:020000040000FA
:100000007828040000000000EE230000EE2300002A
:10001000EE230000EE230000EE230000EE2300009C
:10002000EE230000EE230000EE230000EE2300008C
:10003000EE2300000A240000EE230000EE2300005F
:10004000EE230000EE230000EE230000EE2300006C
:10005000EE230000E0250000EE230000EE23000068
:10006000EE230000EE230000EE230000EE2300004C
:10007000EE230000EE230000EE230000EE2300003C
:10008000EE230000EE230000EE230000EE2300002C
:10009000EE230000EE230000EE230000EE2300001C
:1000A000EE230000EE230000EE230000EE2300000C
:1000B000EE230000EE230000EE230000EE230000FC
:1000C000EE230000EE230000EE230000EE230000EC
:1000D000EE230000EE230000EE230000EE230000DC
:1000E000EE230000EE230000EE230000EE230000CC
:1000F000EE230000EE230000EE230000EE230000BC
:10010000EE230000EE230000EE230000EE230000AB
:10011000EE230000EE230000EE230000EE2300009B
:10012000EE230000EE230000EE230000EE2300008B
:10013000EE230000EE230000EE230000EE2300007B
:10014000EE230000EE230000EE230000EE2300006B
:10015000EE230000EE230000EE230000EE2300005B
:10016000EE230000EE230000EE230000EE2300004B
:10017000EE230000EE230000EE230000EE2300003B
:10018000EE230000EE230000EE230000EE2300002B
:10019000EE230000EE230000EE230000EE2300001B
:1001A000EE230000EE230000EE230000EE2300000B
:1001B000EE230000EE230000EE230000EE230000FB
:1001C000EE230000EE230000EE230000EE230000EB
:1001D000EE230000EE230000EE230000EE230000DB
:1001E000EE230000EE230000EE230000EE230000CB
:1001F000EE230000EE230000EE230000EE230000BB
:1002000070280000000000008344550050000000EA
:1002100000277800000006000A0000008444520015
:100220004F5000003E007800000006000A00000069
:1002300084535700414200000080FD00000006008A
:100240000A000000834E4900500000000E87E800BD
:10025000000006000A000000C4545500434B000093
:100260001E27780010079800000006000C00000010
:10027000C4535700415000009E1F7800000F7800C3
:100280004F007800000006000E000000C44F56002A
:1002900045520000002778001E0090000000060074
:1002A0000C000000C3524F0054000000801F780073
:1002B0001E0090003E0F78004F27780000000600D7
:1002C00010000000C4504900434B00000000E9004A
:1002D000000040006E007800000006000E000000E4
:1002E000C4504F004B4500000000E90000004000F2
:1002F0000E0040003E0878003E0078000000060036
:1003000012000000C4524F004C4C00000000E900F5
:100310000C003400811F7800821F78008E0040009E
:1003200081004000911F7800010178000000E90081
:1003300000800900C21078004F0F78004F0178004C
:10034000CF0078003E007800000006002600000084
:10035000C43F4400555000000000B00001003200CE
:1003600000277800000006000E000000823E5200C8
:10037000801F78003E007800000006000A000000A0
:1003800082523E00002778004F00780000000600EF
:100390000A00000082524000002778007FB89700D2
:1003A000000006000A0000008140000010007800F4
:1003B0000000060008000000C24340001040780022
:1003C0000000FB00000006000A000000C121000040
:1003D0003E0878003E007800000006000A00000099
:1003E000C24321001E4878003E0078003E0078009D
:1003F000000006000C000000812B00003E004000C1
:100400000000060008000000C22B2B00811F7800AE
:10041000BE0078003E0040001E8F4800CF007800EC
:100420000000060010000000864E450047415400C1
:10043000450000000000EA00000006000C0000007B
:10044000812D00003E0010000000060008000000A2
:10045000C22D2D00811F7800BE0078003E001000E4
:100460001E8F1800CF00780000000600100000006A
:1004700082322A004100DD00000006000800000072
:1004800082342A004200DD0000000600080000005F
:1004900082322F004180DE000000060008000000CC
:1004A00082342F004280DE000000060008000000B9
:1004B00082303C004F80DE00000006000800000093
:1004C000C2303D000000B000010032000080EF00AB
:1004D0000080EA00000006000E000000C2303E006E
:1004E0000000B000020032000080EA004F80DE0011
:1004F000000006000E000000C2553C003E00100047
:100500000000EF00F2FF3900000006000C000000C0
:10051000C13C00003E0010000000EF00ECFF350081
:10052000000006000C000000C13D00003E00680015
:100530000000EF00E6FF3200000006000C000000A3
:10054000C13E00003E0010000000EF00E0FF3C0054
:10055000000006000C000000C34E4F0054000000D5
:100560000000B000DAFF32000000EF0000000600DB
:100570000E000000C2552A00811F78003E00B8001E
:10058000CF007800000006000C000000C12A000027
:10059000811F78003E80B900CF007800000006007F
:1005A0000C000000C5552F004D4F4400821F7800FD
:1005B000811F7800000178001E00780011000900FA
:1005C0000280D800010F7800CF0078004F0178003A
:1005D000000006001A000000C6552A002F4D4F00EB
:1005E00044000000821F7800811F7800000178001D
:1005F0003E0078001E00B800110009004288D800B3
:10060000010F7800CF0078004F017800000006004D
:100610001E000000C52A2F004D4F4400821F7800A5
:10062000811F7800000178003E0078001E80B9002C
:10063000110009004208D800010F7800CF007800AF
:100640004F017800000006001C000000C42F4D0080
:100650004F440000821F7800811F7800000178005D
:100660001E007800110009000200D800010F780078
:10067000CF0078004F017800000006001A0000004B
:10068000C12F0000811F780080007800F1FF070073
:1006900001F0A300010039008100EA00801F78000A
:1006A0003E00780000F0A300010039000000EA00DD
:1006B0004100DD00810050004F007800CF0078003D
:1006C0000500390000F0A300020031000000E8003E
:1006D000000006000000E9000000060030000000F5
:1006E000C34D4F0044000000DAFF07003E007800D1
:1006F000000006000C000000C22A2F00811F7800B5
:1007000080007800C5FF0700E1FF37000000060009
:100710000E000000C453510052540000831F7800A3
:10072000821F7800811F78000027EB00010820005D
:100730001E8140000211B8000200E10001003900F2
:100740001E8F40008100D100F9FF39001E01E80032
:100750001E11B8000010E100010031001E0FE8007A
:10076000CF0078004F017800CF0178003E0078007C
:100770000000060032000000C34D41005800000098
:100780001E00E10002003C003E0078000000060070
:10079000620747000000060012000000C34D490038
:1007A0004E0000001E00E100F9FF35003E00780019
:1007B000000006000E000000C3414200530000008C
:1007C0000000B00001003B000000EA00000006004D
:1007D0000E00000083414E00440000003E00600017
:1007E000000006000A000000824F52003E00700028
:1007F000000006000800000083584F00520000006F
:100800003E006800000006000A000000C3415300DB
:10081000480000000000B0000800320004003B0067
:100820000080EA00008009001E8FD100030037001D
:100830000000E900008009001E0FD0003E00780093
:10084000000006001E000000C34C530048000000DA
:100850000000B000F9FF3200F5FF3B000080EA0025
:10086000008009001E0FD100F4FF370000000600D1
:1008700016000000C3524F004C0000000000B00002
:10088000EEFF320004003B000080EA000080090017
:100890001E0FD300E9FF37000000E90000800900C7
:1008A0001E0FD200E5FF3700000006001E0000000A
:1008B00083434F004D0000000080EA000000060066
:1008C0000A000000C32B430021000000811F7800B4
:1008D000BE00780010C840003E007800CF007800CD
:1008E0000000060012000000C32D4300210000009C
:1008F000811F7800BE00780010C810003E0078000C
:10090000CF0078000000060012000000C22B21007A
:10091000811F7800BE007800108840003E007800FB
:10092000CF0078000000060010000000C22D21005A
:10093000811F7800BE007800108810003E0078000B
:10094000CF0078000000060010000000C4464900F7
:100950004C4C0000821F7800811F78003E01780017
:10096000BE0078000201E90002800900805878008A
:100970003E007800CF0078004F01780000000600AC
:100980001C000000C5434D004F564500821F7800F3
:10099000811F78003E0178009E001100BE007800A3
:1009A000050039000000E90009003300008009005B
:1009B00031597800060037000201400081004000F4
:1009C0000000E90002003300008009004161780066
:1009D0003E007800CF0078004F017800000006004C
:1009E00030000000C44D4F0056450000821F7800C3
:1009F000811F78003E0178009E001100BE00780043
:100A0000050039000000E9000B00330000800900F8
:100A1000311978000800370002014000020140004F
:100A200081004000810040000000E9000200330026
:100A300000800900412178003E007800CF00780056
:100A40004F01780000000600340000008449440093
:100A50004C4500000140FE00000006000A000000B6
:100A600085534C00454550000040FE000000060044
:100A70000A000000C8535F0054414D00504F4E0023
:100A80000027780000802000000006000E00000013
:100A9000C6535F00574F5200440000000027780003
:100AA00000862000000006000E000000C8535F0012
:100AB000464F52004D41540000277800008A200024
:100AC000000006000E000000C549540052583100D5
:100AD0000027780000902000000006000C000000B5
:100AE000C55445004C454300002778004090200045
:100AF000000006000C000000C6434E00544954009C
:100B000050000000002778006090200000000600E0
:100B10000E000000C3504100440000000027780090
:100B200020912000000006000C000000C33E490098
:100B30004E000000002778004091200000000600D1
:100B40000C000000C94D45004D5F44004550540065
:100B50004800000000277800609120000000060097
:100B600010000000CB4D45004D5F5000524748003B
:100B700045524500002778008091200000000600C3
:100B800010000000CA414400525F4300524541003A
:100B90005445000000277800C091200000000600A6
:100BA00010000000C5535400415254000027780043
:100BB00000922000000006000C000000C554450013
:100BC0004D5053000027780040922000000006009E
:100BD0000C000000C5544100434845000027780040
:100BE00060922000000006000C000000C84D450087
:100BF0004D5F480045524500002778008092200054
:100C0000000006000E000000CA5354004F505F0061
:100C1000464F52005448000000277800A092200060
:100C20000000060010000000C4454F004C4E0000BC
:100C300000277800E0922000000006000C00000071
:100C4000C3454F00460000000027780000932000B5
:100C5000000006000C000000C442410053450000A3
:100C60000027780020932000000006000C00000000
:100C7000C55354004154450000277800409320009C
:100C8000000006000C000000C5455200524F520003
:100C90000027780060932000000006000C00000090
:100CA000C9545F005355530050454E0044000000A6
:100CB00000277800C093200000000600100000000C
:100CC000C8505200494F520049544500002778004F
:100CD000E0932000000006000E000000CA494E000C
:100CE000505554005F4649004C45000000277800ED
:100CF000009420000000060010000000C7505200C1
:100D0000475F50004E54000000277800409F2000AD
:100D1000000006000E000000C54445005054480085
:100D200000277800E03F21000E0050004180DE00E7
:100D30000000060010000000C65244004550540058
:100D40004800000000277800403021000080570054
:100D50004180DE000000060012000000C750520073
:100D6000474845005245000082FF070000277800F1
:100D7000801F78003E0078002000B000100078004E
:100D8000002778004F00780010007800000006006F
:100D90001C000000C83E5000524748004552450024
:100DA00074FF070000277800801F78003E0078005D
:100DB00087FD0700002778004F0078002000B00072
:100DC00083FD0700000006001C000000C4454D0024
:100DD00049540000002778000027780030012000E7
:100DE000D2FD07002BFD070000277800100120002E
:100DF000CEFD07003E007000D9FD07000000B000E6
:100E00003E0078001E00320037FF07001000780017
:100E10000000B0003E0078000E003200002778008D
:100E200080BB200030FF070069FD07000027780025
:100E3000A0002000BDFD07000000B0003E007800CB
:100E40000300320000277800E00220000100370094
:100E500000000600002778000000B0003E00780087
:100E600007003200A1FF07002008B00053FD070073
:100E700094FD07000000B0003E007800F9FF32004A
:100E8000002778000000280090FF07000027780066
:100E9000801F78003E00780000277800100078005E
:100EA000801F78003E00780049FD07000027780089
:100EB0002022200010007800002778000020200069
:100EC0003E0060000000B0003E00780003003200E9
:100ED0000027780000002000050037000027780078
:100EE000402220003AFD070000277800F0FF2F0085
:100EF0000000B0003E007800ECFF320000277800D0
:100F00004F007800002778004F00780030FD070080
:100F100000000600A6000000C45052004740000038
:100F200079FF0700811F7800821F7800BE007800DB
:100F30001000A7001500370002C02F0002816000DA
:100F40001010E10011003A00100190001E10E100A5
:100F50000E003A004000B000E13FB20000804000C7
:100F6000C108DE00008040000001EB000000A60088
:100F7000B0007800304178000000A600B000780092
:100F8000020F7800010078000500370022032000DE
:100F90001E0978001181BA00020F78001100BA0012
:100FA0004F017800CF007800000006004C000000E0
:100FB000C45052004721000053FF0700811F7800F2
:100FC000821F7800BE00780002C02F0002816000FE
:100FD0001010E10003003A00100190001E10E10023
:100FE000060032001000A6002800070002C02F00F3
:100FF000029860001E107800110007004000B00049
:10100000E13FB20000804000C108DE0000804000E7
:1010100062074700BE0078003E0178000000A6008D
:1010200001187800025878000000A6000118780026
:101030003E0078004F017800CF00780000000600E5
:10104000811F7800821F7800831F7800841F78003A
:10105000B00078002203200030097800F30F200050
:101060001101BA003182BA000218780004587800E1
:101070001101BA003182BA000458780002187800D1
:101080008301E900F6FF310031003700811F78004D
:10109000821F7800831F7800841F780021042000BD
:1010A000020E2000911F780091087100B0007800B6
:1010B00022042400023B880022032000300978002B
:1010C0008108BB0052052000323B8800A20A2000A4
:1010D000323B880061E7A80000000000000000002B
:1010E0007300200012002400023B8800831F780058
:1010F000F301200030017800304278008208BB0004
:101100008498BB0030427800300178008208BB0030
:101110008498BB008301E900F6FF310052052000EE
:10112000323B8800A20A2000323B880061E7A80019
:10113000000000000000000061E7AF00FEFF370084
:10114000CF0178008301E900E6FF31004200F90099
:1011500041602000008010004F027800CF0178002D
:101160004F017800CF00780000000600E00000008A
:10117000C4505200472C0000FBFE070045FC07004E
:1011800044FC0700002778000000200000277800BA
:10119000200020009DFC070001FF070086FF0700DC
:1011A000000006001C000000CB7370005F73790024
:1011B0006E63700072672100D3FE07001000A60066
:1011C000B2FF07001000A0003E00780000000600FB
:1011D00032000000C44845005245000086FE07006A
:1011E00010007800000006000C000000C53E48001A
:1011F0004552450080FE070075FC07000000060010
:101200000C000000C2432C00F4FF07000027780008
:101210001000B000F7FF070072FC07000000060096
:1012200010000000C12C0000ECFF07000027780030
:101230002000B000EFFF070065FC0700000006007B
:1012400010000000CA7370005F636F006D7069006A
:101250006C6500000FFC07000EFC070030FF070064
:10126000801F78003E007800002778003E0068006C
:10127000002778007FB8970000277800F00320004F
:101280003E0060001000B000002778003000200011
:10129000F0FC0700F8FB070091FC07003E0010007F
:1012A0004100DD0059FC0700002778004F0078005E
:1012B00000277800000420003E0060000000B0001D
:1012C0003E00780031003200A7FE070000277800BA
:1012D0000000200000277800200020004BFC0700C1
:1012E0005CFC0700EBFB070000277800F0FF2F00F5
:1012F0008EFC07000000B0003E0078000D003200B8
:10130000801F78003E0078003E00780000277800BB
:1013100070002000002778004F0078004180DE0038
:1013200000277800000028003E00700092FF0700B0
:10133000150037008CFE0700002778000000200011
:10134000002778002000200030FC07002FFC070059
:10135000801F78003E0078000027780020002000E1
:10136000002778004F00780083FF0700801F780077
:101370003E00780000277800000020000027780059
:101380004F0078007CFF070017003700C1FB070003
:10139000C0FB0700E2FE070077FF07000027780088
:1013A00000002000002778002000200017FC070024
:1013B000B8FB0700B7FB0700D9FE070041FC070098
:1013C000ADFB0700002778006000200057FC0700F5
:1013D0003E0060000000B0003E007800EBFF3200ED
:1013E0003E0078003E00780000000600E6000000A5
:1013F0004249460000277800000B200000277800B3
:10140000000020005CFF0700002778008007200014
:1014100000277800E003200057FF0700002778002E
:101420002003200000277800F0FF2F0052FF070064
:101430004DFE07000000060026000000C773700084
:101440005F73610075740000801F78003E007800B3
:10145000801F78003E0078008EFB07008DFB0700A0
:1014600000277800000020000027780020002000DE
:10147000F8FB0700AAFE07003E007800002778006E
:101480004F007800002778004F0078000027780090
:10149000500020008DFB070000277800500020003E
:1014A0008AFB0700EBFB0700801F78003E007800F6
:1014B00000277800F0002000E5FC070000277800F6
:1014C0004F00780000277800F0FF2F00E0FC0700B5
:1014D0003E00400000277800400020008BFB070002
:1014E000002778004000200088FB070000277800D4
:1014F000000020000027780020002000D5FB070016
:10150000ADFE0700000006008E00000044454C00C0
:101510005345000000277800700320000027780062
:10152000F0FF2F0014FF07000FFE0700C6FF0700A3
:101530000DFE07000000060018000000445448009B
:10154000454E000008FE0700BFFF07000000060030
:101550000C00000044434100534500000027780080
:1015600000002000002778000027780000002000FD
:1015700000277800601B200036FF070000000600EF
:1015800018000000424F46000027780000002000AD
:1015900000277800A01C20002EFF070000277800FD
:1015A00000002000002778004029200029FF0700C4
:1015B00090FF0700000006001C00000045454E009B
:1015C000444F4600D3FF0700000006000A00000059
:1015D00047454E004443410053450000D0FD0700FD
:1015E0004180DE005CFB07000000B0003E00780098
:1015F00025003200002778003000200033FB070070
:10160000002778003000200030FB07003E0070000B
:101610000000B0003E00780008003200801F780013
:101620003E007800D0FD070087FF07000027780004
:101630004F0078001000B100020037003E00780033
:101640003E007800002778009EFB07000000B000F5
:101650003E007800E7FF32003E0078000027780067
:101660000000200000277800001C2000F9FE070081
:10167000002778000000200000277800E0102000FC
:10168000F4FE07000200370000277800F0FF2F006B
:1016900000000600640000004542450047494E0036
:1016A000B1FD0700000006000A00000045554E008D
:1016B00054494C004FFF07000027780040002000ED
:1016C00012FB070000277800400020000FFB0700F6
:1016D0005DFF0700000006001800000045574800A5
:1016E000494C450043FF0700000006000A000000C7
:1016F00046524500504541005400000085FF070058
:10170000002778004000200000FB07000027780039
:1017100040002000FDFA07004BFF07000000060014
:101720001A00000042444F0000277800000020000B
:101730000027780080132000C6FE07008AFD0700FE
:10174000002778000000200000277800601B2000A0
:10175000C0FE070000277800000020000027780066
:10176000601B2000BBFE07000000060026000000F2
:10177000452B4C004F4F5000002778000000200000
:1017800000277800001C2000B2FE07000027780028
:101790000000200000277800C01F2000ADFE0700D9
:1017A000002778000000200000277800001C20009F
:1017B000A8FE07000027780000002000002778001E
:1017C00060142000A3FE070000277800000020001E
:1017D00000277800601420009EFE07000027780094
:1017E00000002000002778008028200099FE0700D4
:1017F000002778000000200000277800C02A200081
:1018000094FE0700ABFF07000027780000002000CF
:1018100000277800E01020008EFE070000277800E7
:101820000000200000277800E010200089FE07005B
:101830000000060064000000C74C490054455200F7
:10184000414C000000277800800720000027780026
:101850000070220048FE070000277800801F7800F3
:101860003E0078000027780040FF2F00F8FB0700BB
:101870000002B000002778004F00780000277800B1
:1018800040002000F2FB07003BFE07004AFE070075
:101890000000060030000000444C4F004F50000094
:1018A0000027780010002000E6FF0700B2FF0700C5
:1018B00000000600100000008149000000277800A9
:1018C0007FB89700000006000A000000814A00006F
:1018D000002778005FB89700000006000A000000AB
:1018E000814B0000002778003FB8970000000600F9
:1018F0000A000000854C450041564500002778004D
:101900004F0078004F007800801F7800801F78001B
:101910003E007800000006001400000084455800D6
:10192000495400000000060008000000C2435200B5
:1019300000277800D000200026FD0700002778004F
:10194000A000200023FD0700000006001200000098
:10195000C44245004C4C0000002778007000200075
:101960001CFD0700000006000E000000C5535000DB
:1019700041434500002778000002200015FD0700C4
:10198000000006000E000000C65350004143450011
:101990005300000070FA07000000B0003E0078001D
:1019A00008003200F3FF07001000B10000277800A4
:1019B000C4FA07000000B0003E007800F9FF3200D2
:1019C0003E0078000000060022000000C4545900C8
:1019D0005045000000277800C1FA07000000B00061
:1019E0003E0078002F0032001000B100801F780008
:1019F0003E0078000027780070FA07000027780082
:101A0000F00F20003E00600000277800ADFA0700CC
:101A100020FA07000027780030002000C3FA0700F2
:101A20003E0070000000B0003E0078000900320067
:101A30003E007800002778004F0078003E007800D4
:101A40000027780000002000801F78003E0078000A
:101A50000B0037000027780000277800D000200016
:101A6000B2FA07000000B0003E0078000300320028
:101A70003E007800AEFF070001003700D5FC0700EC
:101A80001000B000002778004F0078000027780091
:101A90008CFA07000000B0003E007800D2FF320050
:101AA00069003700002778004F80DE000000B0009A
:101AB0003E00780064003200801F78003E0078000D
:101AC000F4F90700F3F9070015FD07000027780077
:101AD0004F0078000000EA00002778000000B00006
:101AE0003E00780014003200801F78003E0078002D
:101AF0000027780080FF2F0055FB070000277800A3
:101B000000277800D000200088FA07000000B0000D
:101B10003E007800030032003E00780084FF07009A
:101B200001003700ABFC0700002778004F00780069
:101B30001000B10002003700CFF907003E00780026
:101B400000277800801F78003E0078000000B00079
:101B50003E0078001100320000277800002778004E
:101B6000D000200071FA07000000B0003E007800AD
:101B7000030032003E0078006DFF070001003700CF
:101B800094FC0700002778004F0078001000B10097
:101B9000801F78003E007800010037003E0078008A
:101BA0000027780000002000002778002000200097
:101BB00016FA0700B7F90700B6F90700D8FC0700C6
:101BC000002778004F007800002778000000B00060
:101BD0003E00780014003200801F78003E0078003C
:101BE0000027780000277800F00F20003E006000FA
:101BF0000027780000277800D00020004BFA07006B
:101C00000000B0003E007800030032003E00780083
:101C100047FF0700010037006EFC0700002778002F
:101C20004F0078001000B1000027780025FA070067
:101C30000000B0003E007800A7FF32003E007800B0
:101C40003E0078003E0078003E0078003E007800BC
:101C50000000060046010000C5434F00554E5400E9
:101C6000002778001000B00083F90700D3F90700BF
:101C700000277800F00F20003E0060000000060002
:101C800016000000C92D5400524149004C494E0035
:101C9000470000000027780011FA070000277800AD
:101CA0003000200089F9070000277800300020006C
:101CB00086F907001000B1003E004000BFF90700A0
:101CC000002778000002200018FA07003E0060009C
:101CD0000000B0003E007800020032001000B100A9
:101CE000ECFF37000000060034000000C34249004A
:101CF0004E0000000027780020002000D8FB0700DD
:101D0000B3F907000000060010000000C54F4300B3
:101D100054414C000027780080002000D0FB0700D1
:101D2000ABF907000000060010000000C7444500A2
:101D300043494D00414C000000277800A0002000DE
:101D4000C7FB0700A2F90700000006001200000010
:101D5000C34845005800000000277800000120001B
:101D6000BFFB07009AF90700000006001000000002
:101D7000C7434F004E564500525400001000B000BB
:101D8000002778000000200042F907008BF90700C7
:101D90000027780000277800B0022000E3F9070050
:101DA0000000B0003E007800070032003E007800DE
:101DB000801F78003E0078001000B00000277800F7
:101DC0004F0078000C00370000277800D002200078
:101DD000D6F907000000B0003E007800060032008F
:101DE000801F78003E0078001000B00000277800C7
:101DF0004F0078001000B100801F78003E0078008E
:101E0000002778006DF907000003B1000027780073
:101E10004F80DE000000B0003E0078000400320079
:101E20003E00780000277800F0FF2F0035003700D3
:101E3000002778000027780090002000C1F90700F3
:101E40000000B0003E007800060032007000B100D3
:101E50000027780000277800A0002000ADF90700D7
:101E60000200370000277800000020000000B000CA
:101E70003E007800040032003E0078000027780021
:101E8000F0FF2F001F0037000027780074FB0700C9
:101E9000100078009FF907000000B0003E007800B5
:101EA00015003200801F78003E007800801F780007
:101EB0003E0078006AFB070010007800AEF90700CA
:101EC000002778004F0078001000B000002778004D
:101ED0004F007800E8F80700801F78003E00780087
:101EE0003E004000002778004F007800002778006F
:101EF00000002000030037003E0078000027780033
:101F0000F0FF2F000000B0003E007800BCFF320060
:101F1000002778004F0078000000B0003E007800F5
:101F200005003200801F78003E0078000000EA00C3
:101F3000002778004F00780000000600E80000004D
:101F4000C23C23000027780000002000DAFA0700D6
:101F500024F9070000277800801F78003E007800F1
:101F60004F80DE00002778004F00780014FA070049
:101F7000000006001C000000C4484F004C44000054
:101F8000CDFA0700002778001000B0000027780085
:101F90001000B0000027780030002000CBF80700C8
:101FA00006F9070000277800F00F20003E006000CF
:101FB00000277800E0052000FAF9070073FA07000F
:101FC00000277800FDF8070000277800F00F2000B8
:101FD0003E0060001000B00000277800E0052000FF
:101FE000F0F90700ABF80700FEF807001000B0009A
:101FF000FCF807000000060042000000C1230000BA
:1020000017FB07001000780068F907009AF807002E
:102010000003B0000027780000277800900320001C
:1020200048F9070000277800700020003E0060009B
:102030003E004000D2FF0700000006002200000022
:10204000C2235300EEFF07000027780044F9070081
:102050000000B0003E007800FAFF320000000600E9
:1020600012000000C4534900474E000089F80700E1
:102070000000B0003E007800030032000027780026
:10208000D0022000BEFF070000000600160000007E
:10209000C2233E003E0078003E00780086FA07002A
:1020A000EFFE0700000006000E000000C12E000039
:1020B000A4FF07000027780000022000B0FF0700FF
:1020C000E0FF0700E9FF0700F2FF070041FE0700FD
:1020D0000000060016000000C13F0000100078005C
:1020E000F3FF0700000006000A000000C2552E00A2
:1020F000002778000000200092FF070000277800EA
:10210000000220009EFF07003E0078005AF80700FA
:10211000CCFF0700DFFF07002EFE070000000600CF
:102120001C000000C4574F0052440000801F78007C
:102130003E00780059FA07000027780000002000D0
:1021400054F80700A7F807000027780000002000D7
:10215000B7FA07009EF8070000277800000020006B
:10216000B9FA07009AF807006CFA07001000780027
:1021700070FA0700100078003E0040000027780049
:10218000801F78003E0078001000B0000027780023
:102190001000200067FA0700DDF90700002778002B
:1021A0004F00780085F8070000277800F00F200026
:1021B0003E00600000277800801F78003E00780015
:1021C000002778003000200040F807000027780042
:1021D0007AF807003E0040001000B00081F80700C8
:1021E000002778004F00780000277800B5F8070036
:1021F00028F807000027780030002000CBF80700FF
:102200003E0070000000B0003E0078000A0032007E
:102210003E00780000277800F0FF2F0000277800AC
:1022200083FA07006AF807000027780086FA07009B
:1022300067F807002E003700002778000027780095
:10224000D0002000B9F807000000B0003E00780080
:10225000070032003E00780000277800F0FF2F00D2
:102260000027780072FA070059F8070020003700AD
:1022700000277800801F78003E0078000027780053
:1022800090002000A9F80700002778007FB8970089
:102290000027780000022000A4F807003E0070002C
:1022A000002778004F007800002778007FB897005B
:1022B0009EF807003E0070000000B0003E0078006D
:1022C0000300320000277800F0FF2F0008003700DD
:1022D0000027780010002000002778003000200040
:1022E000FAF7070079F907000027780000002000BE
:1022F0000000B0003E007800A0FF32003E007800F1
:10230000002778004F0078003E00780000000600AB
:10231000F8000000C127000000277800000220001C
:1023200082FF07000027780024F807000000B000B3
:102330003E007800CE003200801F78003E0078001A
:102340001AFA070000277800801F78003E00780006
:102350002000B00010007800002778004F007800BF
:1023600010007800002778007FB8970000277800D9
:102370000027780011F807003E0040001000B00070
:102380000027780040002000D0F7070000277800E1
:1023900040002000CDF70700BEF70700BDF707009B
:1023A000DFFA070000277800F0F32F003E006000FE
:1023B000002778004F007800B6F707000027780064
:1023C000F00F20003E006000B2F70700FBF70700A7
:1023D00000277800F00F20003E00600053F807004F
:1023E0000000B0003E007800350032001000B00060
:1023F0000027780060002000B4F70700A5F7070069
:1024000050F807000000B0003E00780029003200BC
:10241000A0F707000027780080FF2F000CF90700C5
:102420009CF70700E5F7070040F807000000B00040
:102430003E0078001C0032001000B0000027780039
:1024400060002000A1F7070092F707003DF80700A1
:102450000000B0003E007800100032000027780035
:102460003000200099F707008AF70700D3F707002C
:102470002EF807000000B0003E0078000400320093
:102480001000B00000277800F0FF2F000200370096
:1024900000277800000020000200370000277800A5
:1024A000F0FF2F0002003700002778000000200016
:1024B0000200370000277800F0FF2F0002003700ED
:1024C0000027780000002000801F78003E00780080
:1024D000801F78003E0078003E0078003E007800C3
:1024E000002778004F007800002778004F00780020
:1024F0000000B0003E0078001F0032000027780086
:102500004000200071F7070062F707000DF8070090
:102510000000B0003E0078000F003200801F7800FD
:102520003E00780000277800000020000027780097
:1025300020002000B5F7070056F7070055F7070001
:1025400077FA0700002778004F007800002778000E
:1025500000002000070037003E0078003E007800B1
:102560003E0078003E0078003E00780000277800AA
:10257000F0FF2F003A0037003E0078003E00780060
:102580003E007800801F78003E007800801F7800B1
:102590003E0078003FF707003EF70700002778006D
:1025A000000020000027780020002000A9F7070085
:1025B0005BFA070037F7070036F707003E007000A8
:1025C0000000B0003E00780017003200A1F70700BD
:1025D000002778004F007800002778004F0078002F
:1025E000002778004000200038F707000027780017
:1025F0004000200035F7070026F7070025F7070001
:1026000047FA070000277800F0F32F003E00600033
:1026100000277800600020002CF7070000277800D2
:10262000000020000E003700002778004F007800DF
:10263000002778004F0078003E0078003E007800C8
:102640003E0078003E0078003E00780000277800C9
:102650003E0068000027780000277800F0FF2F0078
:102660000000B0003E00780053FF32000300370046
:10267000002778003E006800002778000000060070
:10268000B8010000C44649004E44000022FF070084
:1026900000F70700FFF607003E0070000000B000E2
:1026A0003E00780015003200FAF60700F9F6070040
:1026B0001BFA0700801F78003E0078000027780092
:1026C0003E006800002778004F007800002778005F
:1026D000F00320003E0060001000B00000277800EA
:1026E00030002000DBF70700E3F607007CF7070067
:1026F0003E0010004100DD0044F707000000060026
:1027000040000000415B000000277800000020002E
:1027100059F907002EF70700000006000E00000020
:10272000C15D000000277800F0FF2F0052F907007C
:1027300027F70700000006000E000000C13A000065
:10274000002778000002200078FE070086F90700C5
:1027500000277800000020000027780020002000DB
:102760002AF7070011F9070000277800801F78007A
:102770003E0078002000B0001000780000277800AC
:102780007FB897001000780032F707007AFA070048
:1027900075F90700002778007FB897000CF707004D
:1027A000002778004F0078002000B00008F70700ED
:1027B0000027780001F7070000277800F0032000C9
:1027C0003E0060001000B000801F78003E007800DE
:1027D000002778002000B000F8F6070000277800F6
:1027E000F00F20003E006000AAF607001000B000C5
:1027F000F2F60700002778008000200014F8070098
:10280000002778007FB897001000B10000277800FB
:10281000000C20003E0070003E00400056FA070009
:102820003000B000002778004F0078003000B10081
:10283000002778002AF707000000B0003E0078006B
:1028400016003200801F78003E00780000277800D4
:102850002000B000D9F6070000277800F00F200014
:102860003E0060008BF607001000B000D3F60700B2
:102870000027780080002000F5F707000027780087
:102880003000200091F60700CCF607000027780002
:10289000F00F20003E006000DFFF37003E007800B0
:1028A0003E00780000277800F0FF2F00F2F80700C4
:1028B000C7F607001AF90700A6F80700C4F60700D4
:1028C00000000600C6000000413B00000027780021
:1028D00060002000002778000000200026FA070092
:1028E00035FA07000027780000002000E2F8070012
:1028F000B7F607000AF9070096F8070010007800FD
:102900003E0010000000B0003E0078000E003200D3
:102910000027780030002000DDF80700ACF6070043
:102920007EF8070010007800D9F807002000B000FA
:10293000A7F607007FF8070010007800D4F807001A
:102940004000B000A2F607000000060044000000AE
:10295000C87370005F7461006368650000277800C9
:102960004F007800002778004F007800002778009B
:102970003000200055F6070000277800801F7800FF
:102980003E0078008000B00091F607000027780034
:102990004F007800A000B0008DF607000000060090
:1029A0006E000000C6544100434845003A00000054
:1029B00063FF070009FA0700A2FB07000027780061
:1029C0000000200018FA070000277800000020000F
:1029D00015FA0700002778000000200012FA07000F
:1029E00000277800000020000FFA07000027780079
:1029F000000020000CFA07000027780000002000EB
:102A000009FA07000027780000002000002778005E
:102A1000804A21000FFA0700000006003E00000077
:102A2000C9545F0045584500435554004500000017
:102A300000277800801F78003E007800A000B000DA
:102A400010007800002778004F0078008000B00068
:102A500010007800801F78003E007800801F78000A
:102A60003E0078000000060026000000C8545F0009
:102A7000414A4F00555445008DF807000027780063
:102A8000801F78003E007800100078000027780052
:102A9000F0FF2F00002778007FB897004CF6070062
:102AA000801F78003E0078004CF80700002778006F
:102AB0001000780028F607000000B0003E00780003
:102AC000350032000027780030002000FFF50700B5
:102AD000F0F5070095F607000000B0003E00780012
:102AE000070032003E0078003E0078003E0078008B
:102AF0003E00780000277800F0FF2F002500370007
:102B0000002778001000780000277800500020008F
:102B1000EEF5070079F607000000B0003E007800EF
:102B2000140032000027780030002000E7F507008D
:102B30004000B00026F60700801F78003E007800B5
:102B400000277800002778004F00780020F6070063
:102B500000277800F0FF2F00CEF507002000B0001E
:102B60001BF607001AF6070000277800F0FF2F0079
:102B700008003700801F78003E0078003E00780093
:102B8000002778004F0078004000B0000027780050
:102B90000000200013003700801F78003E007800FE
:102BA00000277800002778004F00780008F607001B
:102BB00000277800F0FF2F00B6F507002000B000D6
:102BC00003F607000027780000002000B1F5070099
:102BD0004000B000FEF50700FDF507000027780073
:102BE000F0FF2F000000B0003E007800AFFF320081
:102BF000002778004F007800002778004F00780009
:102C0000F3F5070000000600D0000000C8545F0084
:102C10004143540049564500801F78003E0078002B
:102C20000027780010002000D5F607000027780064
:102C300000002200DBF60700002778004F00780034
:102C40006000B000E2F5070000000600220000006E
:102C5000C9545F0050455200494F440045000000F0
:102C6000801F78003E0078000027780010002000C8
:102C7000C3F607000027780000002200C9F607000D
:102C8000002778000000EA00002778007FB897004E
:102C90006000B000CEF507004180DE00C9F70700F4
:102CA000100078003E00400000277800F0FF270069
:102CB0003E006000002778004F0078002000B00040
:102CC000C3F50700000006003E000000C8545F0086
:102CD00052455400495245009FF507000000B000DE
:102CE0003E0078003D003200F1F707000027780031
:102CF000801F78003E0078001000780000277800E0
:102D0000F0FF2F00002778007FB89700B0F507008C
:102D1000801F78003E007800B0F707005DF50700DF
:102D20005CF507001000780000F607000000B00016
:102D30003E00780015003200801F78003E007800C9
:102D4000002778000000200052F507006000B00066
:102D50009FF50700002778004000B00010007800C1
:102D6000002778004F00780099F5070000277800C9
:102D70000000200047F507004000B00094F5070070
:102D800000277800F0FF2F000B00370010007800BC
:102D900071F507000000B0003E007800040032002A
:102DA0004000B0000027780000002000020037003B
:102DB00000277800F0FF2F000000B0003E007800F0
:102DC000D6FF32003E007800002778004F007800E0
:102DD000002778004F0078007DF50700000006000E
:102DE0008C000000C57370005F2E6700002778001C
:102DF0004F007800002778004F00780025F5070085
:102E000024F5070046F8070000277800F00F20009F
:102E10003E006000801F78003E0078003E00780091
:102E20001CF507001BF507000027780000002000B4
:102E3000002778007FB897001000B00000277800C6
:102E40003000200003F607000BF50700A4F507008B
:102E50003E0010004100DD006CF5070000277800FF
:102E60004F00780004F50700801F78003E007800CE
:102E700001F50700801F78003E0078000000EA009E
:102E8000D4FA070000000600E0000000C5544C0022
:102E90004953540051F70700100078002EF5070041
:102EA0000000B0003E00780070003200002778007B
:102EB000A000B00010007800F6F407008000B00019
:102EC000100078000027780000002000002778001C
:102ED000200020005FF50700EEF40700EDF4070086
:102EE0000FF807003E0078000027780080072000D8
:102EF0008EF507000000B0003E007800F1FF3200C0
:102F00000027780000002000002778002000200023
:102F100050F50700DFF40700DEF4070000F80700B3
:102F2000801F78003E0078003E007800002778007F
:102F30004F00780000277800002778000008200064
:102F40003E0060000000B0003E0078000900320042
:102F500000277800F00320003E0060000000EA0037
:102F60009CFA070083FA070000277800F0FF2F0083
:102F700002003700002778003E0068000000B00023
:102F80003E007800DEFF320035F7070010007800C1
:102F9000801F78003E00780067FB070093FF070062
:102FA0000B707200696F720069746500203A20002E
:102FB00000277800100078004DFC07002000B000CA
:102FC000002778004000B00010007800002778004B
:102FD0004F80DE000000B0003E0078000B003200A1
:102FE00082FF07000D70650072696F0064697100EF
:102FF000756520003A2078000000EA002CFC0700EC
:103000007AFF0700026D7300110037003E00780060
:1030100000277800100078004F80DE000000B0002C
:103020003E0078000600320070FF070009494E009C
:1030300041435400495645002065200004003700F4
:103040006AFF0700074143005449560045204500E8
:10305000002778004F00780001F70700DCF4070034
:1030600033FA07002000B0008BFF37000000060095
:10307000F400000047434F004D5049004C4500000C
:10308000A5FC070083F4070082F407003E007000EF
:103090000000B0003E0078000900320076F407001E
:1030A000E8F90700E7F90700002778000000200092
:1030B000002778002092200066F8070010003700F3
:1030C0003E0078003E0078000027780030002000A5
:1030D000EFF60700BEF4070090F607001000780036
:1030E000EBF607002000B000B9F4070091F60700E6
:1030F00010007800E6F607004000B000B4F40700C6
:10310000000006004A000000495B43004F4D50009C
:10311000494C45005D0000007FFC07005DF407009E
:103120005CF407003E0070000000B0003E00780034
:103130000200320047F80700100037003E00780018
:103140003E0078000027780030002000D0F607000D
:103150009FF4070071F6070010007800CCF6070016
:103160002000B0009AF4070072F607001000780003
:10317000C7F607004000B00095F407000000060005
:103180003E000000C7455800454355005445000027
:10319000801F78003E007800801F78003E00780095
:1031A0000000060012000000C12200000027780085
:1031B00040002000B0F60700D5F50700EAF607004A
:1031C00000277800F00F2000002778000000200082
:1031D0000000060018000000422E220000277800A0
:1031E0000000200000277800206F210019F8070058
:1031F000EEFF07000000060012000000012800009A
:1032000000277800200020009BF60700C0F507008B
:10321000000006000E000000C22E5300C0F607009A
:103220004DF407000000B0003E0078001C003200A2
:103230000027780000002000801F78003E00780002
:10324000002778001000B000002778007FB89700B2
:103250003E0010001DF4070095FB070000277800D2
:103260004F0078001000B00000277800801F780021
:103270003E00780007F40700A6F40700B8F4070042
:103280000000B0003E007800EDFF3200002778001B
:103290004F0078003E0078003E00780006003700BE
:1032A000D2FE07000C5069006C652000766964004E
:1032B0006520210020207800000006005400000056
:1032C00049494D004D454400494154004500000026
:1032D00036F6070000277800801F78003E0078004F
:1032E0002000B00010007800002778004F00780020
:1032F00010007800E7F30700E6F3070008F707007F
:1033000000277800F0F72F003E00600000277800CB
:1033100040002000FDF30700002778004000200057
:10332000FAF3070024F70700000006003800000049
:103330004644490052454300540000001BF6070074
:1033400000277800801F78003E0078002000B00041
:1033500010007800002778004F00780010007800F7
:10336000CCF30700CBF30700EDF607000027780049
:10337000F0FB2F003E006000002778004000200096
:10338000E2F307000027780040002000DFF3070089
:1033900009F707000000060036000000C5414C0098
:1033A0004C4F5400002778000000B0003E00780029
:1033B0000500320000277800000020009AF707007F
:1033C0001000B100F7FF37003E0078000000060053
:1033D0001C000000C44C4F00414400002CF60700C4
:1033E000100078000000B0003E00780002003200BB
:1033F0003E007800F501370034F607001000780031
:10340000801F78003E007800002778001000200020
:103410002EF60700EEF30700C0F507001000780055
:10342000801F78003E007800C2F507001000780089
:10343000801F78003E007800FDF50700100078003E
:10344000801F78003E007800FFF50700100078002C
:10345000801F78003E007800B0F50700DCF307001D
:103460000027780000002000B2F50700D8F307001D
:1034700001F60700100078000027780018F4070014
:103480000000B0003E007800B6003200002778004F
:10349000200020002BF407000000B0003E00780060
:1034A000A100320000277800200220001FFB070047
:1034B000EBF90700002778003000200083F30700B5
:1034C00000277800F00F20000CF4070071F30700CC
:1034D00003F407003E0060000000B0003E007800EA
:1034E0002C003200801F78003E007800801F78009A
:1034F0003E00780060F3070097F307000000B0007B
:103500003E0078001700320000277800002778007E
:1035100000102000F9F307000000B0003E00780022
:1035200008003200002778007FB89700A3F3070057
:103530000027780080002000C5F407003E0040000E
:1035400007003700002778007FB897009BF307003B
:1035500049F3070008F70700002778000000200063
:1035600003003700002778007FB8970093F3070027
:1035700041F307001000B000002778004F007800EA
:103580001000B000002778004F0078001000B10054
:10359000C8FF37003E00780088F307000027780056
:1035A0000027780020022000E0F307000000B000B0
:1035B0003E0078002A0032003E007800801F78002C
:1035C0003E00780064F307000000B0003E00780081
:1035D00004003200002778000000200026F30700D6
:1035E000E5F607002BF307002AF307004CF6070067
:1035F0000027780000F02F003E00600000277800D0
:103600004F0078003E004000002778004000200076
:103610002EF3070000277800400020002BF307005E
:1036200065F6070094F50700100078000027780081
:1036300030002000BDF307000000B0003E0078001D
:10364000020032003E0078003E007800002778003B
:103650004000200088F50700B5F40700310037006E
:1036600079F50700100078000000B0003E007800F7
:10367000030032003E00780000277800D0002000D0
:1036800004F3070000277800F00F20009BF30700E9
:103690000000B0003E00780021003200801F78005A
:1036A0003E007800F4F207002BF307000000B000A2
:1036B0003E007800150032000027780000277800CF
:1036C000001020008DF307000000B0003E007800DD
:1036D00007003200002778004F00780000277800AC
:1036E000800020005AF407003E004000060037002A
:1036F000002778004F007800DFF207009EF60700F1
:103700000027780000002000020037000027780022
:103710004F007800D8F207001000B0000100370019
:103720003E0078000E0037000027780000022000DD
:103730007EFA070010007800002778001090220021
:103740007AF307000000B0003E0078000400320069
:10375000002778002000200047F5070074F40700D8
:10376000EB0037003E007800EBFA0700C9F20700D3
:10377000C8F207003E0070000000B0003E00780074
:103780005F0032003CF50700100078000000B00038
:103790003E00780024003200BEF20700BDF20700B0
:1037A000DFF50700B4F207003E007800002778003C
:1037B000000820003E0060000000B0003E007800DD
:1037C00002003200A3F6070016003700B1F207002E
:1037D000B0F20700D2F50700801F78003E007800A5
:1037E000002778003E006800002778004F0078002E
:1037F00000277800F00320003E0060001000B000B9
:10380000002778003000200092F307009AF20700AA
:1038100033F307003E0010004100DD00FBF207001B
:103820005BFE0700350037009AF2070099F20700A7
:10383000BBF5070090F207003E00780000277800F3
:10384000000C20003E0060000027780000042000EB
:1038500036F307000000B0003E007800110032008F
:103860003E0078003E00780000277800200020000D
:1038700007F50700D6F20700A8F40700100078004B
:1038800003F507002000B000D1F20700A9F40700FB
:1038900010007800FEF407004000B000CCF20700F2
:1038A000160037007BF207007AF207009CF507004C
:1038B000801F78003E007800002778003E006800F6
:1038C000002778004F00780000277800F0032000E0
:1038D0003E0060001000B00000277800300020009B
:1038E0005CF3070064F20700FDF207003E001000E1
:1038F0004100DD00C5F2070025FE07008400370007
:103900003E00780065F4070000277800ABF207005E
:103910000000B0003E0078007B0032005DF207003E
:103920005CF2070015F9070060F207003E0078001E
:103930005EF207003E007800002778009FF2070043
:103940000027780010022000F2F207000000B0000B
:103950003E007800080032003E007800C6F4070000
:10396000100078000000B0003E0078000100320036
:10397000B4F7070063003700002778008FF20700D4
:103980000027780000277800B0022000E7F2070047
:1039900039F2070000277800D0022000E3F2070088
:1039A0003E0070003BF207001000B00083F20700F9
:1039B0000027780010022000D6F207003E006000C9
:1039C0000000B0003E0078003E00320031F20700F7
:1039D0000000B0003E0078003700320077F20700A8
:1039E000A5F40700100078000000B0003E00780049
:1039F00027003200801F78003E0078000027780002
:103A00000027780000402000BCF207000000B00052
:103A10003E0078000E0032000027780040002000B1
:103A20008BF30700002778004F007800002778000C
:103A3000D0022000BDF2070000277800100020000F
:103A40003E006000000BB0000BF207000E003700D4
:103A50007CF707000027780000042000002778008A
:103A60004F00780000277800D0022000AFF2070056
:103A700000277800000320003E0060003E00100098
:103A800000277800E0032000BBF50700090037009D
:103A900000277800B0022000A4F207000000B00068
:103AA0003E007800020032003E0040000100370076
:103AB0003E001000020037003E0078003E00780013
:103AC000100037003E0078003E00780000277800A4
:103AD000100020006EF407003DF207000FF407000D
:103AE000100078006AF407002000B00038F20700E8
:103AF00010F407001000780065F407004000B000E3
:103B000033F20700020037003E0078003E007800E4
:103B10004DF40700100078005DF4070010007800F5
:103B20003E0070000000B0003E00780050FE320001
:103B30007BF407004F80DE000000B0003E007800FC
:103B40000E003200002778004000200050F40700EB
:103B50001FF20700F1F30700100078004CF4070093
:103B60002000B0001AF20700F2F3070010007800FE
:103B700047F407004000B00015F207000027780066
:103B80004F00780030F4070011F20700002778009A
:103B90004F00780026F407000DF207000027780098
:103BA0004F007800E3F3070009F2070000277800D0
:103BB0004F007800D9F3070005F2070000277800CE
:103BC0004F00780041F4070001F2070000000600F2
:103BD00000040000C6435200454154004500000067
:103BE0007EF5070017F707005FF40700E9F3070009
:103BF00000277800801F78003E007800F4F107006D
:103C0000002778004F0078002000B000F0F1070096
:103C1000002778004000200000277800F0FF2F00E8
:103C200055F50700002778000000200000277800E5
:103C3000F007200050F507005FF5070000000600C0
:103C400038000000C87370005F646F0065733E0049
:103C5000D0F3070000277800801F78003E0078002E
:103C60002000B00010007800002778004F00780096
:103C7000100078000027780000002000002778005E
:103C80004F00780000277800400020008FF10700E7
:103C900000277800400020008CF107000027780002
:103CA000000020000027780020002000D7F1070046
:103CB000C1F40700002778004000200000277800AA
:103CC0004F00780000277800400020008FF10700A7
:103CD00000277800400020008CF10700B6F40700B0
:103CE00035F507000027780000002000E2F3070008
:103CF000B7F10700000006009400000045444F00A3
:103D000045533E000027780000002000002778007F
:103D100020E221004FF5070000000600120000001D
:103D2000C856410052494100424C450084FA070000
:103D3000ABFF07003CF50700C5FF070000000600C9
:103D400012000000C8434F004E535400414E54002F
:103D50007BFA0700BBF60700002778006000200010
:103D6000002778000000200003F5070012F5070087
:103D70000027780000002000BFF3070094F107003F
:103D80000000060022000000C653540052494E00B5
:103D9000470000006AFA070037F10700A9F607009C
:103DA000A8F60700002778006000200000277800B0
:103DB00000002000F0F40700FFF40700002778005F
:103DC00000002000ACF3070081F1070000000600AE
:103DD00026000000C5564C004953540073F30700F9
:103DE00000277800801F78003E0078002000B00097
:103DF00010007800002778004F007800100078004D
:103E000024F1070023F1070022F1070021F1070048
:103E100043F40700801F78003E0078003E007800E1
:103E2000002778004F00780000277800F00320007A
:103E30003E0060000000EA00E6F60700CDF607004D
:103E400014F1070013F1070000277800000020009C
:103E500000277800200020007EF1070030F40700E2
:103E60000CF107000BF107003E0070000000B000ED
:103E70003E0078000400320076F107000027780049
:103E800000002000040037003E0078003E0078006B
:103E900000277800F0FF2F000000B0003E007800FF
:103EA000D7FF32003E0078003E0078000000060098
:103EB00070000000C34B4500590000008BF3070061
:103EC000002778001000B0003CF107000140FE0020
:103ED000F0F0070039F10700EEF007003E00100097
:103EE0000000B0003E007800F8FF3200E9F0070063
:103EF0003E0040002000B00030F10700801F780035
:103F00003E0078001000B000002778002BF1070079
:103F10001000B00000277800F00720003E0060008D
:103F2000D5F007002FF10700002778004F00780038
:103F30000000060042000000C5494E004B455900F4
:103F40006AF30700002778001CF1070000277800BB
:103F50000027780030002000DCF007001000B000DF
:103F600020F107001000B10000277800F0072000C2
:103F70003E0060003E0040002000B0000FF107004E
:103F80000000060028000000C84B450059424F00C1
:103F90004152440055F307001000B000002778009C
:103FA0001000B10005F10700BAF0070003F10700A7
:103FB0003E0010000000B0003E0078000600320015
:103FC00000277800FDF007003E0040001000B00020
:103FD000FAF0070002003700002778003E00680072
:103FE0000000060030000000C64558005045430060
:103FF0005400000000277800F00F20003E00600011
:104000000027780000002000002778003000200002
:10401000AEF00700F3F007009EF007001000B000BC
:104020009CF00700002778000002200049F20700FA
:10403000A2FF07000027780000277800F001200089
:1040400040F1070093F0070000277800F0072000F8
:1040500030F107003E0060008EF007000027780076
:104060009000200031F107003E007000002778002A
:104070004000200095F00700D0F0070000277800EE
:104080004000200091F0070022F107003E00600090
:104090000000B0003E0078004700320000277800A2
:1040A000002778009000200020F107000000B000F9
:1040B0003E007800180032003E00780000277800AB
:1040C00000022000002778008000200000277800F0
:1040D000400020007DF00700B8F0070000277800BE
:1040E000801F78003E0078000027780070002000D4
:1040F0003E0060003E0010000027780030002000E5
:1041000072F00700002778004F0078003E00100092
:10411000A4F10700020037000027780010002000FB
:10412000801F78003E00780000277800801F78000C
:104130003E0078000027780026F30700002778006B
:104140003000200061F007009CF007001000B00074
:1041500000277800400020005CF00700A1F0070075
:10416000002778003000200058F007000027780072
:1041700092F007003E0040009AF007000027780008
:104180004F007800002778004F0078001000B10041
:1041900000277800CBF007000000B0003E00780058
:1041A000DFFF32003E0078003E00780000277800F4
:1041B000000020004F00370000277800002778001B
:1041C000F0072000D9F0070032F007000027780040
:1041D00080002000D5F007003E0070002DF00700A1
:1041E00000277800C0012000D0F007003E007000DA
:1041F000002778004000200034F007006FF007002F
:10420000B7F007003E0060000000B0003E007800FC
:10421000140032003E0078001EF0070067F007002F
:1042200000277800100020003E00100000277800D2
:104230003000200025F007006AF007000027780012
:1042400080002000E3F20700CAF50700002778008D
:1042500080002000DFF20700002778000000200027
:104260002400370000277800002778003000200065
:10427000AEF0070007F0070000277800D00020000C
:10428000AAF007003E00700002F007008DF0070062
:104290003E0070000000B0003E0078000B003200CD
:1042A000002778003000200008F007000027780081
:1042B00042F007001000B0003E00400049F0070047
:1042C00000277800F0FF2F000A0037000027780051
:1042D000A000200095F00700A1F007000000B0004A
:1042E0003E007800010032009BF5070000277800AF
:1042F000000020000000B0003E0078004CFF3200BB
:104300003E0078003E0078000000060094010000A6
:10431000C4515500495400000F3021000027780097
:10432000000020000027780053F2070028F0070063
:1043300057F2070026F007004FF207001000780040
:1043400005F007000000B0003E00780015003200C4
:10435000002778004F80DE000000B0003E007800AB
:10436000040032003E00780000277800A0032000FF
:104370000B003700002778002000200071F00700B4
:104380000000B0003E0078000300320000277800F3
:104390002002200002003700002778008002200061
:1043A0000200370000277800E003200089F20700B0
:1043B000B3F1070000277800CBF107001000780068
:1043C0000000B0003E0078000300320000277800B3
:1043D000F00520000200370000277800E0042000EC
:1043E00004FF070052F50700002778003000200086
:1043F000A8EF070000277800F0EF07003E0040001C
:104400001000B000F7EF0700002778000000200040
:10441000A0EF0700F3EF07001000B000B2F10700B3
:10442000100078000000B0003E0078000800320064
:10443000002778003001200066F20700E7FB070044
:10444000002778001001200062F207000100370009
:10445000E2FB07000EF20700100078000000B00039
:104460003E007800A00032000E4021009EF10700BF
:10447000100078000000B0003E0078000900320013
:10448000C4FE07000000B0003E00780002003200C9
:104490008AFE07003E007800002778000000200018
:1044A0000200370000277800F0FF2F000000B00066
:1044B0003E007800EDFF3200EFF1070010007800B9
:1044C00000277800F0FF2F0018F007000000B00070
:1044D0003E00780020003200B4F107000027780089
:1044E000801F78003E0078002000B00010007800A7
:1044F000002778007FB897001000780065EF07006C
:1045000064EF070063EF070062EF07000027780001
:10451000000020000027780020002000CDEF0700D9
:104520007FF20700CBEF0700002778007FB89700E5
:10453000A7EF0700002778004F0078002000B000A8
:10454000A3EF070016F20700002778000000200004
:10455000C9F107009EEF070024FA0700052A2A0088
:104560002A2A20004DF10700BDF5070019F50700C4
:1045700000F50700C6F1070010007800002778005A
:104580000027780010002000E8EF07000000B000CE
:104590003E0078000A00320014FA0700183A2000A2
:1045A000496E730074727500637469006F6E200049
:1045B000494E43004F4E4E0055452000217478006F
:1045C000002778000027780020002000D7EF0700A0
:1045D0000000B0003E0078000A00320003FA070035
:1045E000193A2000496E7300747275006374690093
:1045F0006F6E2000494D4D0045444900415445002F
:104600002021780000277800002778003000200063
:10461000C6EF07000000B0003E0078000B0032003B
:10462000F2F907001B3A200050524F00424C45005F
:104630004D45200050696C006520640065205200E3
:1046400045544F0055522000210D5400002778009A
:104650000027780040002000B4EF07000000B00001
:104660003E0078000B003200E0F907001D3A200000
:1046700050524F00424C45004D45200050696C009F
:104680006520640065732000444F4E004E45450090
:1046900053202100002778000027780040002000E8
:1046A000A8EF07000000B0003E00780008003200CC
:1046B000CEF907000C3A20004552520045555200F1
:1046C000206E6F0020696C0079F60700010037004A
:1046D0003E007800A0F4070095F40700002778005A
:1046E000F0FF2F000F00370063F107001000780083
:1046F00074EF07000000B0003E00780007003200B1
:1047000000277800F0042000B2F1070000277800AD
:10471000B0042000AFF1070085F4070000277800FF
:10472000000020000000B0003E00780002FF3200D0
:1047300000277800000020000000B0003E00780054
:10474000F5FE3200000006001E020000C5414200D6
:104750004F5254000E40210097F2070000277800C6
:10476000000020000027780058F1070018EF07002C
:10477000002778004EF1070015EF070000277800AA
:10478000E6F0070012EF0700EAF0070010EF07005D
:1047900067F4070095F90700262A2A002A2A200034
:1047A000494E54004552520055505400494F4E0056
:1047B000204C6F006769630069656C006C652000C0
:1047C000284142004F5254002920210058F407008C
:1047D00061F40700D0FE0700000006000027780003
:1047E0006003200000277800801F78003E007800DA
:1047F00010007800002778004F007800002778002C
:1048000010002000BFF0070041F00700F0EE0700A5
:104810000040060000277800600320000027780091
:10482000801F78003E007800100078000027780094
:104830004F0078000027780010002000E1F007000A
:1048400033F0070000277800400820000027780098
:10485000801F78003E007800100078000027780064
:1048600070FF2F003E006000002778004F007800A6
:10487000D7EE07000EF107001000780011EF0700D7
:104880000000B0003E0078008C00320096F0070077
:10489000100078000000B0003E0078002C003200CC
:1048A00091F0070000277800801F78003E00780014
:1048B000100078001000B100002778000027780071
:1048C0004F007800C2EE0700FEEE07000000B000C7
:1048D0003E0078001E00320004F107000027780037
:1048E000B6EE07001000B00000277800F0072000A7
:1048F0003E00600067EE07001000B000AFEE07005A
:1049000064EE070009EF07000000B0003E007800E9
:10491000030032003E0078003E0078000C003700B3
:1049200000277800D0002000002778003000200009
:1049300066EE070000277800A0EE07003E0040006A
:104940002000B000A7EE07004BEE0700A5EE070021
:10495000DEF0070010007800A0F0070010007800DB
:10496000002778000000B0003E00780051003200BF
:1049700048EE070047EE070010007800DFEE070062
:104980000000B0003E007800450032008DF00700C6
:10499000100078003FEE07002000B0001000780003
:1049A000002778004F80DE00801F78003E007800EE
:1049B0003E00100000277800000024003E00600048
:1049C000002778004F0078003E007000E4EE0700FA
:1049D0000000B0003E007800170032000027780089
:1049E00010007800B9F0070079EE07000027780082
:1049F0000000280027EE07002000B000C4EF0700E9
:104A0000002778004280BF00002778007FF89700D9
:104A1000004EB20042E0B7003E0078001DEE0700F5
:104A200003F8070042E0B7003E00780019EE0700E7
:104A3000A6F0070066EE070062F00700811F78000D
:104A4000821F7800100178009E0078008180E800C5
:104A50001100E0000B003B00210090000000E0008E
:104A60000800320002003B00110010000300370074
:104A7000000041000001EB00A200980000F0A1003E
:104A8000800878003E0078004F017800CF00780061
:104A900020009000002778008AEE0700020037000F
:104AA00000277800F0FF2F000000B0003E007800E3
:104AB000AFFF32003E0078003E00780083F0070030
:104AC0001000780000277800200020008BEE0700FF
:104AD0000000B0003E007800370032004EF00700C2
:104AE00000277800801F78003E00780010007800D2
:104AF000002778004F0078002000B00010007800F8
:104B0000E4ED0700E3ED07003E0070000000B00098
:104B10003E007800260032000027780000002000C8
:104B2000002778003CF0070000277800801F7800FD
:104B30003E00780026EE0700002778004F0078003E
:104B40002000B00022EE0700F4EF0700100078000C
:104B50000000B0003E00780012003200002778000C
:104B6000F00720003E006000002778004F0078002A
:104B70000027780000F82F003E0060003E00400053
:104B8000002778004F0078003E007800BAED07005B
:104B9000801F78003E007800801F78003E0078007B
:104BA000020037003E0078003E0078000200370027
:104BB0003E0078003E00780005EE07000040060049
:104BC000002778006003200000277800801F78000D
:104BD0003E00780010007800002778004F00780031
:104BE0000027780060222000F4ED070000277800FD
:104BF0004008200000277800801F78003E007800E1
:104C00001000780000277800F07F2F003E00600041
:104C1000002778004F007800EDED0700ACEF0700AB
:104C200000277800801F78003E0078002000B00048
:104C300010007800002778004F00780010007800FE
:104C400094ED070093ED07003E0070000000B000F7
:104C50003E007800020032004DF9070046003700A0
:104C60003E0078003E007800002778001000B10078
:104C70000000B0003E0078003200320000277800CB
:104C8000002778003001200028EE070081ED0700A2
:104C9000002778001001200024EE07003E0070007D
:104CA0000000B0003E0078000700320000277800C6
:104CB000300120001DEE07000CF007002008B000B6
:104CC000C8ED07001E00370008F007000027780035
:104CD000BAED07001000B00000277800F0072000B0
:104CE0003E0060006BED07001000B000B3ED070060
:104CF00068ED07000DEE07000000B0003E007800F0
:104D0000040032003E0078003E0078003E0078004B
:104D10000B00370065ED0700002778003000200009
:104D20006AED070000277800A4ED07003E00400070
:104D30002000B000ABED07004FED0700A9ED070024
:104D40000D003700002778003E006800002778003B
:104D5000603A2200B0EF070000277800801F78003B
:104D60003E0078009AED0700002778004F00780099
:104D70002000B00096ED070095ED0700004006000A
:104D80001C030000D15449004D455200315F5500CD
:104D900041525400315F49004E49540000277800C9
:104DA00000022000002778004074200088ED0700F2
:104DB00000277800F0CF270000277800201020007F
:104DC00083ED070000277800000028000027780006
:104DD000401020007EED07000027780040042000EE
:104DE000002778008022200079ED07000027780056
:104DF00000002000BDEF070075ED070000277800D8
:104E000080002800002778000022200070ED0700B5
:104E10000027780000402000002778002022200092
:104E20006BED0700002778008080200000277800C5
:104E30004009200066ED07000027780000002000F0
:104E400030EF070062ED070000000600660000007A
:104E5000C55445004D504F005AEF07001000780030
:104E60000140FE000BED070056EF07001000780030
:104E7000002778003000200014ED07003E001000ED
:104E80009EED07000000B0003E007800F4FF320005
:104E90003E0078003E007800000006002800000078
:104EA000C5464F0052544800D0F70700CA0D4500D0
:104EB0006E747200657A200064616E0073206C006D
:104EC00065206D006F6E64006520640075204600EB
:104ED0004F525400480D0D00202020002020430098
:104EE0006F70790072696700687420006A706200F0
:104EF0002E666F00727468000D0D2000204D690051
:104F000063726F0020464F0052544800202070000A
:104F10006F7572002050490043323400464A0D003C
:104F200020566500727369006F6E2000312E3200CA
:104F3000322020006475200031362F0031312F00DF
:104F400032303100340D20002068740074703A0053
:104F50002F2F6A0070622E00666F720074682E0038
:104F600066726500652E6600722F0D0020206A00B3
:104F700070625F00666F720074684000796168005B
:104F80006F6F6700726F750070732E00636F6D0036
:104F90000D0D200051756500206C650020464F0006
:104FA0005254480020736F006974200061766500D8
:104FB000632054004F4921000D0D0D000000060034
:104FC00092000000C6464F005247450054000000C2
:104FD000D1F40700AFEC0700AEEC07003E00700014
:104FE0000000B0003E0078001D003200A9EC070070
:104FF000A8EC0700002778000000200000277800B8
:105000002000200013ED0700A2EC0700A1EC070030
:1050100063EF0700C2EF07000EED0700E3EE0700A5
:1050200000277800801F78003E007800E8EC070039
:10503000002778004F0078002000B000E4EC070063
:1050400000277800F00F200000277800F0FF2F00E5
:1050500045EF0700D8EF070057F0070002003700C0
:105060003E0078003E007800000006005600000078
:10507000CE5445004C4543004841520047454D0041
:10508000454E54000AEF070000277800801F780083
:105090003E0078001000780000277800F0FF2F0015
:1050A000002778007FB89700C9EC0700801F7800C0
:1050B0003E0078000027780080BB20008AEE0700C1
:1050C000C3EC0700002778004F0078000027780025
:1050D0004F007800BEEC070000000600380000001A
:1050E000C94445004D41520052414700450000006F
:1050F000A03A210020A0B7000F3021000E4021006F
:105100005FEE07000027780000B02000002778003D
:10511000000020000FEE070000277800100020009C
:10512000F9EE0700AAEC07000027780080FF2000B6
:1051300030F0070019FF070007F307000027780089
:1051400000002000002778000010200074EF070006
:1051500050EC07004FEC070000277800000020000B
:105160000027780020002000A8EC070049EC070089
:1051700048EC07006AEF0700801F78003E007800C7
:1051800000277800F00F2000E8EC070000277800E7
:105190004F00780000277800F0FF2F00E3EC0700B5
:1051A0003E0060000000B0003E007800EAFF3200E0
:1051B00038EC070037EC0700F9EE070035EC070084
:1051C000002778005000200040EC0700D7EC0700D3
:1051D00030EC070000277800500020003BEC07006F
:1051E000D2EC07003E0060000000B0003E007800F6
:1051F000050032003E0078003E007800002778006D
:10520000F0FF2F006900370022EC070021EC0700B7
:1052100000277800000020000027780020002000F0
:105220008CEC07003EEF07001AEC07000000B0000E
:105230003E0078000A0032003E0078003E00780010
:1052400000277800000020000027780020002000C0
:1052500080EC070000277800000020005300370092
:10526000801F78003E007800801F78003E007800A4
:1052700008EC070007EC0700002778004F007800D3
:10528000002778004F00780072EC070001EC07005F
:105290004F80DE000000B0003E0078000C003200BD
:1052A0003E0078003E0078000027780000002000D3
:1052B000002778002000200066EC07000027780017
:1052C0000000200000277800F0FF2F003400370096
:1052D000F0EB07000027780070002000FBEB0700D0
:1052E00092EC0700EBEB070000277800700020002D
:1052F000F6EB07008DEC07003E0060000000B000F8
:105300003E0078000A0032003E0078003E0078003F
:10531000E6EB07003E007800E4EB07003E00780073
:1053200000277800F0FF2F00002778001C003700CE
:10533000D8EB0700D7EB070000277800000020001B
:10534000002778002000200042EC0700F4EE070060
:10535000D0EB07000000B0003E0078000E003200E5
:105360003E0078003E0078003E0078003E00780065
:10537000002778000000200000277800200020008F
:1053800034EC070000277800000020000027780098
:10539000F0FF2F00020037000027780000002000F7
:1053A0000000B0003E007800B7FF32000000B000FF
:1053B0003E00780081FF3200B6EB0700B5EB070036
:1053C000FAED070000277800801F78003E00780083
:1053D000FFEB0700002778004F0078002000B000A6
:1053E000FBEB0700ABEB0700AAEB0700CCEE0700D6
:1053F000801F78003E00780000277800100420000D
:105400004AEC0700002778004F007800002778005A
:1054100050CC240045EC07003E0060000000B000C6
:105420003E007800200032000027780000002000B5
:105430000027780020002000F4EB070095EB070020
:1054400094EB0700B6EE0700801F78003E0078005E
:10545000002778005004200034EC07000027780073
:105460004F00780000277800E03424002FEC07007C
:105470003E0060000000B0003E00780007003200EF
:10548000002778000000200000277800200020007E
:10549000DEEB07003EF70700020037003E00780011
:1054A0003E007800020037003E0078003E007800A1
:1054B00021F207007CFE070027F1070096FB07009A
:1054C00000000600FFFFFF00FFFFFF00FFFFFF00DF
:00000001FF
